:100000000C94D9020C9411030C9411030C94110359
:100010000C9411030C9411030C9411030C94110310
:100020000C9411030C9411030C94E3250C94B52645
:100030000C94E0200C9411030C9411030C94110304
:100040000C9411030C9411030C9411030C941103E0
:100050000C9411030C9468210C9411030C9411035B
:100060000C9411030C9411030C9411030C941103C0
:100070000C9411030C9411030C9411030C941103B0
:100080000C9411030C9411030C9411030C941103A0
:100090000C9411030C9411030C9411030C94110390
:1000A0000C9411030C9411030C941103B005B005CA
:1000B000DC05DC0544066F076F076F076206FB0669
:1000C0000C070C07041EFA1D071E4F1E531E531E5D
:1000D0004F1E531E531E281E531E321E3C1E531EFF
:1000E000531E531E531E4F1E531E531E4F1E531E90
:1000F000151E531E531E4C1E4C1E4C1E4C1E4C1ED9
:100100004C1E4C1E4C1E4C1E511E531E041EF71D31
:10011000531E531E531E531E531E531E531E531E57
:10012000531E531E511E531E531E4F1E531E4A1E56
:100130004A1E4A1E4A1E4A1E4A1E4A1E4A1E4A1E7F
:10014000511E222749274128492741289527B827AA
:1001500041280F281E2829001E001F002000210012
:100160002200230024002500260027002D002E0059
:1001700035002A002B0014001A0008001500170093
:100180001C0018000C00120013002F00300031007A
:100190000000390004001600070009000A000B00E7
:1001A0000D000E000F003300340000002800000096
:1001B000E10000001D001B000600190005001100F1
:1001C0001000360037003800E50052004C00E00017
:1001D000E300E20001510000000000002C0001518A
:1001E000E600E400500051004F000000005C3A00BF
:1001F0003B003C003D003E003F004000410042000B
:1002000043004400450001004C000100C35C520063
:10021000C45CC65CC75CC85CC95CCA5CCB5C0100E2
:1002200001000100010000000100500051004F00DA
:1002300001000100010001000100010001000100B6
:100240000000010000000100000001000100BE5C90
:10025000C05CBF5C01000100010001000100010061
:100260000100010001000100010001000000000088
:100270000000010001000100010001000100010077
:10028000000000047F3F1F643214643214783C1E67
:100290001E140A052223252628292A2C2D2F303228
:1002A000333536383A3B3D3E4042434547494A4C58
:1002B0004E5051535557595A5C5E60626466686986
:1002C0006B6D6F71737577797B7D7F81838587898E
:1002D0008A8C8E90929496989A9C9E9FA1A3A5A793
:1002E000A8AAACAEAFB1B3B4B6B8B9BBBCBEBFC1BF
:1002F000C2C3C5C6C7C9CACBCCCDCED0D1D2D2D34A
:10030000D4D5D6D7D7D8D9D9DADADBDBDBDCDCDC5D
:10031000DCDCDDDDDDDDDCDCDCDCDCDBDBDBDADA20
:10032000D9D9D8D7D7D6D5D4D3D2D2D1D0CECDCC97
:10033000CBCAC9C7C6C5C3C2C1BFBEBCBBB9B8B6AC
:10034000B4B3B1AFAEACAAA8A7A5A3A19F9E9C9A37
:1003500098969492908E8C8A89878583817F7D7B05
:1003600079777573716F6D6B6968666462605E5CE6
:100370005A5957555351504E4C4A494745434240AC
:100380003E3D3B3A3836353332302F2D2C2A292842
:1003900026252322FFAA7F5540000101010101010A
:1003A000010101020202020202020202030303032C
:1003B00003030303040404040404040505050505FC
:1003C00006060606060707070707080808080909BA
:1003D00009090A0A0A0B0B0B0C0C0C0D0D0D0E0E65
:1003E0000E0F0F0F101011111112121313141415F8
:1003F0001516161717181819191A1A1B1B1C1D1D6C
:100400001E1E1F20202122222324242526262728C1
:1004100029292A2B2C2D2D2E2F30313232333435F1
:10042000363738393A3B3C3D3E3F404142434445F4
:10043000464748494A4C4D4E4F50515354555658D3
:10044000595A5B5D5E5F616264656668696B6C6D7D
:100450006F7072737577787A7B7D7E8082838587F3
:10046000888A8C8E8F91939596989A9C9EA0A2A331
:10047000A5A7A9ABADAFB1B3B5B7BABCBEC0C2C436
:10048000C6C9CBCDCFD1D4D6D8DBDDDFE2E4E7E9F6
:10049000EBEEF0F3F5F8FAFDFF0C0359004D0044C4
:1004A000003600370000000A0359004D0044004B9D
:1004B0000000000403090409023B00020100A0FA45
:1004C00009040000010301010009211101000122BA
:1004D0004000070581030800010904010001030031
:1004E0000000092111010001226D0007058203208F
:1004F000000112010002000000084D596060010077
:100500000102000105010980A101850319012AB733
:1005100000150126B700950175108100C0050C0972
:1005200001A101850419012AA002150126A0029546
:100530000175108100C005010906A10185060507A6
:1005400019E029E7150025019508750181020507C5
:10055000190029EF1500250195F0750181020508A4
:100560001901290595057501910295017503910100
:10057000C005010906A101050719E029E7150025B5
:10058000019508750181029501750881010507191A
:100590000029FF150026FF00950675088100050853
:1005A00019012905950575019102950175039101C0
:1005B000C00011241FBECFEFDAE0DEBFCDBF04B60E
:1005C00003FE18C080911F0390912003A091210386
:1005D000B09122038730904BA740B04B59F4109252
:1005E0001F03109220031092210310922203E0E0D7
:1005F000F8E3099511E0A0E0B1E0E8E0F3E502C01E
:1006000005900D92A03CB107D9F723E0A0ECB1E032
:1006100001C01D92AF31B207E1F70E946B130C9439
:1006200082290C94000081E0089581E008950C94E3
:10063000150308950C9419031F93CF93DF9300D0F3
:1006400000D01F92CDB7DEB749835A836B833091B8
:10065000C30189819A81311114C0662359F0222384
:1006600049F00E94A809182F682F89819A810E9459
:10067000510903C00E947C09182F69817A81812F5A
:1006800004C00E94A80969817A810F900F900F9091
:100690000F900F90DF91CF911F910C94D610FC0119
:1006A000262F408151816281738184810C941C03C7
:1006B00081E00895CF93DF93EC0160E00E944F0347
:1006C000BE01DF91CF910C941A030C941C120C9470
:1006D000181208950E94FB070E9469032FEF84E31C
:1006E0009CE0215080409040E1F700C000000C9455
:1006F0008E210F931F93CF93DF938C0161E00E94B3
:100700004F03EC01B8010E941703882309F44BC082
:10071000B801CE010E94661B882309F444C0B801C9
:10072000CE010E94391F8823F1F1B801CE010E9449
:100730008C1C8823C1F1B801CE010E94951E88232C
:1007400091F1B801CE010E94AA19882361F1F80144
:100750008281882309F1CB358DE5D807C1F050F4AB
:10076000C115FCE5DF0781F0CF3DDC45A9F40E940F
:10077000DF0E19C0CC35EDE5DE0761F0CD35DD4586
:1007800059F40E94220E08C00E946A030CC00E9405
:100790002B0E02C00E942E0EC801DF91CF911F9137
:1007A0000F910C94130380E0DF91CF911F910F9173
:1007B00008950E94C22080E00E949B1B0C94F703C6
:1007C0000E948A1A0E94FA030C94C82008950C947F
:1007D000E60381E008950C94E9030895CF93C82FB0
:1007E0000E94E7038C2F0E94EB03CF91089580E0D5
:1007F0000C94EE030E94951F0C94EE030E94951F2B
:100800009091C201891721F08093C2010C94EE03EC
:100810000895CF93DF93CDB7DEB72B970FB6F8943B
:10082000DEBF0FBECDBF4F83588769877A878B871E
:1008300061110E946E0D9E012F5F3F4F86E0F9010E
:1008400011928A95E9F785E0FE013796D90101906A
:100850000D928A95E1F789819A814C815D81452BC2
:1008600031F09F3F31F491E08F3F19F403C091E0E4
:1008700001C090E090FF09C049815A816B817C8161
:100880008D819E810E948F0C05C0C9010E94580372
:100890008111F2CF2B960FB6F894DEBF0FBECDBFFD
:1008A000DF91CF910895FC01808191810E94EA0936
:1008B0000895CF93882309F495C0C82F8238A1F4F6
:1008C00069E380910201909103010E947D200E94C2
:1008D000900D2FEF81EE94E0215080409040E1F7A1
:1008E00000C0000069E315C08338E1F463E580913E
:1008F0000201909103010E947D200E94900D2FEF34
:1009000081EE94E0215080409040E1F700C000006B
:1009100063E580910201909103010E948820CF91AC
:100920000C94900D8438A1F467E4809102019091B9
:1009300003010E947D200E94900D2FEF81EE94E034
:10094000215080409040E1F700C0000067E4E1CF13
:100950008CEF8C0F813AF8F48C2F0E94591E811174
:1009600041C06C2F80910201909103010E94FD1FF4
:10097000882349F06C2F80910201909103010E941D
:1009800088200E94900D6C2F8091020190910301AC
:100990000E947D20C4CF80E28C0F883048F4C7705D
:1009A00081E001C0880FCA95EAF70E94510DB7CFC8
:1009B000EBE5EC0FE33040F4F0E0EE5AFE4F8081BF
:1009C00090E0CF910C94BB1FC85AC73158F4EC2F5C
:1009D000F0E0EE0FFF1FEC5DFE4F80819181CF9123
:1009E0000C94D11FCF910895882309F44FC0682F2C
:1009F000823859F469E380910201909103010E94C9
:100A00007D200E94900D69E30CC0833891F463E56A
:100A100080910201909103010E947D200E94900D1F
:100A200063E580910201909103010E9488200C945B
:100A3000900D843859F467E480910201909103018C
:100A40000E947D200E94900D67E4EBCF8CEF860F13
:100A5000813A38F380E2860F883048F4677081E08D
:100A600001C0880F6A95EAF70E94570DE0CF8BE529
:100A7000860F833020F480E090E00C94BB1F685A0E
:100A8000673120F480E090E00C94D11F08951F930B
:100A9000CF93DF93182FEB010E945904209741F068
:100AA0008FE99FE00197F1F700C000002197F6CF92
:100AB000812FDF91CF911F910C94F404893319F0A9
:100AC00060E070E002C060E570E00C9447058823A8
:100AD00021F00E94510D0C94900D0895882321F06F
:100AE0000E94570D0C94900D0895CF92DF92EF92D3
:100AF000FF920F931F93CF93DF937C01D62FC72FC5
:100B0000FC011281058102950F700E94470D882318
:100B1000B9F01123A9F08C2F807F803421F080E27E
:100B20008D0F883068F08091CF0282FD09C082E08D
:100B30000E94F00D0E94470D91E0D82ED92601C0E9
:100B4000D12CCC2EC2948FE0C8228C2D90E08C301A
:100B5000910508F0C4C1FC01EA5AFF4F0C94DD284E
:100B60008C2F807FCF70882311F0C295C07F112316
:100B700099F0CC2309F49FC180E28D0F883010F0EA
:100B8000D11104C08C2F0E94510D03C08C2F0E94E4
:100B9000610D0E94900D8FC18D2F0E94F404CC2313
:100BA00009F49DC180E28D0F883038F1DD2329F1F1
:100BB0008C2F0E94670D24C08C2F807FCF708032D5
:100BC00011F0C295C07FDD2319F0D130A1F13DC0F5
:100BD0008091CF0282FF17C0112349F0CC2329F066
:100BE0008C2F0E94510D0E94900D80E065C180E025
:100BF0000E94F404CC2309F472C18C2F0E94570D7B
:100C00000E94900D6CC1112371F0002341F001305E
:100C100031F40E94710D8C2B0E94790D60C10E94ED
:100C2000710D8C2B1DC0002319F0013009F457C140
:100C30000E94860D25C0112321F0063008F04FC117
:100C40000EC0053008F04BC11BC0112361F000231A
:100C500031F0F701858180FF2EC18F7085838C2F45
:100C60000E9467053CC1002359F0D93309F034C113
:100C7000FFEF07EE13E0F15000401040E1F72AC10A
:100C80008C2F0E946E052BC18C2F869586958370C4
:100C900019F0813061F023C1112321F08D2F9C2F99
:100CA000937002C080E090E00E94BB1F20C111231E
:100CB00021F08D2F9C2F937002C080E090E00E9465
:100CC000D11F15C18C2F837009F047C011110BC1C2
:100CD0002D2F229526952770220F220F6D2F6F70D2
:100CE000862F90E0A0E0B0E0022E04C0880F991F8C
:100CF000AA1FBB1F0A94D2F7D4FF10C04FE050E0E8
:100D000060E070E004C0440F551F661F771F2A95EE
:100D1000D2F7409550956095709503C040E050E043
:100D2000BA01C695C695C3708A019B01082B192B81
:100D30002A2B3B2BC901B801C23049F058F4C1300D
:100D400019F00E946708CFC00E945508CCC00E94CD
:100D50007908C9C00E945308C6C0112319F08C2F0E
:100D6000817001C08695882309F4BDC02D2F22957E
:100D700026952770220F220F6D2F6F70862F90E01F
:100D8000A0E0B0E0022E04C0880F991FAA1FBB1F6D
:100D90000A94D2F7D4FF10C04FE050E060E070E05A
:100DA00004C0440F551F661F771F2A95D2F7409540
:100DB00050956095709503C040E050E0BA01C6952B
:100DC000C695C3708A019B01082B192B2A2B3B2B3C
:100DD000C901B801C23049F058F4C13019F00E947D
:100DE0002C0981C00E941A097EC00E943E097BC066
:100DF0000E948D0878C0CF70112339F08C2F0E948B
:100E0000B3088D2F0E9467056EC08D2F0E946E055E
:100E10008C2F0E94D40867C0D23F21F128F4D03F24
:100E200041F0D13FC1F043C0D33F19F1D43F79F035
:100E30003EC0112341F0053008F051C08C2F8F7156
:100E40000E94F9084CC0063008F049C0F7CF8091E5
:100E5000CF0282FF18C0112339F08C2F8F710E94AE
:100E6000B3083DC01123C9F38C2F8F710E94D408A1
:100E700036C0112329F08C2F8F710E949E082FC03D
:100E80000E9499082CC0112349F0CF718C2F0E9429
:100E9000B30863E08C2F0E94D50D21C081E00E9431
:100EA000F00D0230E0F082E00E94F00D18C0112336
:100EB00031F0002391F28D2F0E94590410C00023BD
:100EC00099F2D93349F41FEF27EE33E01150204057
:100ED0003040E1F700C000008D2F0E94F40488EF3D
:100EE0008C0D843020F40E94951F0E94EE03DD20BB
:100EF000C9F00E94430D80FD15C0F70112820E94C7
:100F00003D0D0E94B308C7010E94B3070E943D0D2A
:100F1000DF91CF911F910F91FF90EF90DF90CF90D5
:100F20000C94D408DF91CF911F910F91FF90EF9017
:100F3000DF90CF9008950F931F93CF93DF93EC0131
:100F4000688179818A810E94F5098C010E9450098B
:100F50000E944108B801CE010E947505DF91CF9132
:100F60001F910F910895CF93DF93EC0198818981B0
:100F70002B813C81232B31F08F3F31F481E09F3F67
:100F800019F403C081E001C080E080FD1DC0CE01E6
:100F90000E947903811110C00E94470D8823A1F09F
:100FA0008A81882389F08091CF0282FD0DC082E082
:100FB000DF91CF910C94F00DCE010E949B07CE01E2
:100FC000DF91CF910C945A03DF91CF91089580E087
:100FD00090E00E94BB1F80E090E00E94D11F0E9421
:100FE0006E0D0C94900D80910201909103010E946E
:100FF00093200C94E7070E945E0D0C94F3079295E2
:101000009F70963079F010F4925001C09A5092304F
:1010100068F4803F69F018F4883E40F409C0843FCA
:1010200029F406C0883E20F0813F11F080E0089549
:1010300081E00895FC01808191810E94EA090E946B
:10104000FF070895CF93DF9300D000D01F92CDB754
:10105000DEB70F900F900F900F900F90DF91CF9110
:101060000895CF93DF9300D000D000D0CDB7DEB786
:1010700026960FB6F894DEBF0FBECDBFDF91CF919D
:101080000895089508950C9442080C9443080E9412
:1010900045086093FA017093FB018093FC019093E3
:1010A000FD010C94E7070C9447080F931F930091E0
:1010B000FA011091FB012091FC013091FD01602BA0
:1010C000712B822B932B1F910F910C9447080F9338
:1010D0001F930091FA011091FB012091FC013091C6
:1010E000FD0160237123822393231F910F910C94A0
:1010F00047080F931F930091FA011091FB01209173
:10110000FC013091FD0160277127822793271F91F1
:101110000F910C9447080C9442080E948B0860932E
:10112000F6017093F7018093F8019093F9010C9404
:10113000E70760E070E0CB010C948D080F931F93DC
:1011400041E050E060E070E08A019B0104C0000FC4
:10115000111F221F331F8A95D2F7C901B8011F91B1
:101160000F910C948D080F931F9341E050E060E0C5
:1011700070E004C0440F551F661F771F8A95D2F791
:101180008091F6019091F701A091F801B091F901D9
:101190008A019B01082B192B2A2B3B2BC901B80173
:1011A0001F910F910C948D080F931F9341E050E015
:1011B00060E070E004C0440F551F661F771F8A95DA
:1011C000D2F740955095609570958091F601909179
:1011D000F701A091F801B091F9018A019B01082360
:1011E00019232A233B23C901B8011F910F910C94A5
:1011F0008D080F931F9341E050E060E070E004C061
:10120000440F551F661F771F8A95D2F78091F6010C
:101210009091F701A091F801B091F9018A019B0129
:10122000082719272A273B27C901B8011F910F91C9
:101230000C948D080F931F930091F6011091F70104
:101240002091F8013091F901602B712B822B932BA7
:101250001F910F910C948D080F931F930091F6012D
:101260001091F7012091F8013091F9016023712369
:10127000822393231F910F910C948D080F931F933A
:101280000091F6011091F7012091F8013091F901D8
:1012900060277127822793271F910F910C948D0847
:1012A00008952FE0929F800D1124E82FE695E69592
:1012B000E695877051E001C0550F8A95EAF785E001
:1012C000E89FF0011124EC53FE4F20E030E070E085
:1012D0004081CB01022E02C0969587950A94E2F7D1
:1012E0008170819584278523842781932F5F3F4FC9
:1012F0002530310569F708952FE0929F800D112464
:10130000682F669566956695982F977085E0689F1B
:10131000B001112440E050E080E0FB01E40FF51F34
:10132000EC53FE4F208130E0092E02C03695279500
:101330000A94E2F721703327042E01C0220F0A9489
:10134000EAF7822B4F5F5F4F4530510531F7089523
:10135000BF92CF92DF92EF92FF920F931F93CF93A2
:10136000DF938C01C090F601D090F701E090F80176
:10137000F090F9018091FA019091FB01A091FC019C
:10138000B091FD01C82AD92AEA2AFB2ACFE1D0E090
:10139000D701C6010C2E04C0B695A79597958795E1
:1013A0000A94D2F780FD04C0219790F7B12C07C0B2
:1013B000BC2EB8018C2F0E94E9100197A9F38B2D48
:1013C000DF91CF911F910F91FF90EF90DF90CF9021
:1013D000BF900895CF93DF93EC010E94A809BE014E
:1013E0000E94E910DF91CF9108951F93CF93DF936F
:1013F000EB019091C301992321F0CB010E94EA09EE
:1014000013C0882349F0CB010E94A809182F682F28
:10141000CE010E94510904C0CB010E947C09182F03
:10142000BE01812F0E94E910DF91CF911F91089595
:101430001F93CF93DF93C091FE0116E08091FF01CF
:10144000C81799F0D0E01C9FF0011D9FF00D1124EA
:10145000E050FE4F4081518162817381848195818A
:101460000E9431082196C770E9CFDF91CF911F917B
:101470000895409130025091310260913202709192
:10148000330280913402909135020C943108EF922E
:10149000FF920F931F93CF93DF9380913502829534
:1014A0008F7009F065C080913202882309F460C012
:1014B0008091FE01F090FF01109130020091310205
:1014C000609133027091340291E01F3F09F090E087
:1014D000C0910001D0910101292F96E0E92E8F15CE
:1014E00009F446C06115710521F00F3F21F030E08D
:1014F00003C031E001C0322F90E030FD36C0E89EDD
:10150000F001E99EF00D1124DF01A050BE4F1196AD
:101510003C911197301329C03C91311326C012968B
:101520003C911297311121C013964D915C91149703
:10153000461B570B4C175D07C0F4809135028F7026
:10154000806180933502EB5FFD4F80818F708061F9
:10155000808380E392E00E94B307DF91CF911F91D7
:101560000F91FF90EF900C94180A01968770B7CFF7
:10157000DF91CF911F910F91FF90EF9008959F926F
:10158000AF92BF92CF92DF92EF92FF920F931F9391
:10159000CF93DF93CDB7DEB761970FB6F894DEBF78
:1015A0000FBECDBF8C0185E0F801DE011D960190D4
:1015B0000D928A95E1F7D8011296EC909091300245
:1015C000E09131022091330230913402211531052E
:1015D00031F0EF3F31F481E09F3F19F403C081E027
:1015E00001C080E0B82FB1709B2E80FD47C1D801AB
:1015F0004C9111965C9111971396AD90BC901497F5
:1016000080E3C82E82E0D82EF0903202B501621B32
:10161000730B2091000130910101FF2009F4D9C022
:10162000809135026217730708F095C0282F207F3C
:1016300009F052C05E1313C0491311C0FE2CE11013
:101640000EC08F708061809335020E94390AC601F6
:101650000E94B30780913502F80185834DC1AB2804
:1016600031F05F3F31F481E04F3F19F403C081E076
:1016700001C080E080FD03C081E08E2502C080E0D3
:1016800090E0F82FF170FF2E80FF1CC08091FE01CA
:101690002091FF0136E0821709F40BC190E0389FDA
:1016A000F001399FF00D1124E050FE4F6181561377
:1016B00006C06081461303C06281E61203C0019632
:1016C0008770E9CFFE2CEE2009F416C18091350217
:1016D00081608093350254C05E1306C0491304C074
:1016E000E11002C0F80199C0C8010E941A088823BD
:1016F00061F1EE2051F120913502822F82958F7099
:1017000090E0029774F080913002909131029887B6
:101710008F831986BB86AA862C87CE0107960E94E6
:10172000B30786E0F801A0E3B2E001900D928A953C
:10173000E1F70E94470A0E94390A0AC05E1711F1B8
:10174000C8010E941A0881112CC0C8010E94B30769
:10175000FF24F394D1C0282F207F81F77A2DB98AF6
:10176000A88A6E2D89890E94220880E392E00E9457
:10177000B30786E0D6011D928A95E9F70E94390ADF
:10178000F12CBAC04913DCCFE110DACFF801858320
:10179000C8010E94B30786E0D6011D928A95E9F739
:1017A000ABC0EE2091F220913502822F82958F708E
:1017B00090E002970CF4B5CF809130029091310205
:1017C0009A8389831B82BD82AC822E83CE010196CF
:1017D000A6CF6217730708F044C0FE2CEE2009F470
:1017E000B4CF5E1330C049132EC02091350220FDC6
:1017F00021C0822F82958F70482F50E041155105EE
:10180000C9F0F80125834F30510541F08F5F982FC3
:101810009295907F822F8F70892B8583C8010E94BB
:10182000B30786E0F801A0E3B2E001900D928A953B
:10183000E1F73CC086E0F801A0E3B2E001900D9230
:101840008A95E1F759C0C8010E941A08811169CF31
:1018500080913502816080933502C8010E94B307F0
:101860004BC07A2DB98AA88A6E2D89890E942208D8
:1018700086E0D6011D928A95E9F718C0EE2009F49A
:1018800064CFC8010E941A08F82E882309F45DCF9E
:1018900086E0F801A0E3B2E001900D928A95E1F7AD
:1018A00080E392E00E9453040E94470A0E94390A92
:1018B00023C04D875E878D859E850E94EA09292F6A
:1018C00022952F70223028F49F7039F0811105C0C5
:1018D0000BC0243028F49F7049F4805E883020F0DB
:1018E000C8010E94B3079F2CF92C06C0D801159699
:1018F0009C91907F91F7F8CF8F2D61960FB6F89459
:10190000DEBF0FBECDBFDF91CF911F910F91FF9032
:10191000EF90DF90CF90BF90AF909F9008951F936E
:10192000CF93DF93CDB7DEB72C970FB6F894DEBF19
:101930000FBECDBF4F83588769877A878B879C8777
:10194000CE0107960E94BF0A8823D1F09F81888527
:101950002A853B85232B31F08F3F31F481E09F3F77
:1019600019F403C081E001C080E080FD47C04F81D1
:10197000588569857A858B859C850E9431083EC093
:1019800086E0FE013796DE01119601900D928A9550
:10199000E1F7FF81E8856A857B856115710531F086
:1019A000EF3F31F481E0FF3F19F403C081E001C053
:1019B00080E080FD23C02091FF0130E0C901019645
:1019C000877099274091FE0150E084179507F1F147
:1019D000F983EA837D836C8396E0929FD001939F85
:1019E000B00D1124A050BE4FFE01319601900D9212
:1019F0009A95E1F78093FF010E94180A16E0809102
:101A0000FE019091FF01891771F1189FC001112407
:101A100080509E4F0E94BF0A882329F1E091FE0169
:101A20001E9FF0011124E050FE4F408151816281E0
:101A30007381848195810E9431088091FE0190E03C
:101A40000196877099278093FE01D9CF0E94FB07EA
:101A50001092FF011092FE01E0E3F2E086E0DF0168
:101A60001D928A95E9F72C960FB6F894DEBF0FBE4B
:101A7000CDBFDF91CF911F9108958091560285953A
:101A80008595859508958091560287700895909167
:101A90005602977081E009F480E008958091790200
:101AA000089590917902892B809379020895809509
:101AB0009091790289238093790208951092790296
:101AC000089590917802892B8093780208958095EB
:101AD0009091780289238093780208951092780279
:101AE000089580915702089508950C94740D0C94F4
:101AF000750D9091CF0292FD08C0909157029817F2
:101B000021F0809357020C94770D0895809157022D
:101B1000882329F01092570280E00C94770D0895E5
:101B2000CF93DF93E0910201F0910301809179025C
:101B30008083E0910201F09103019081809178020D
:101B4000892B808380915702882381F0E0910201E4
:101B5000F09103019081892B808380910201909103
:101B600003010E94E71F81110E94860DC0910201AE
:101B7000D091030140E250E066E372E0CE010E94A2
:101B80002D29892B69F080E2FE01A6E3B2E00190E5
:101B90000D928A95E1F7CE01DF91CF910C94A11FB0
:101BA000DF91CF9108950C94740D9091CF0292FD26
:101BB00010C098E0899F90011124262B2093560293
:101BC0000E94B308809156028595859585950C9461
:101BD000D30D0C94B3081092560280E00C94D30DF0
:101BE000209156028095822380935602982F9770F9
:101BF00099F430E0482F082E000C550B24173507B8
:101C000059F09091CF0292FD07C0859585958595F5
:101C10000E94D4080C94EB0D08959091CF0292FB92
:101C2000222720F9281769F080FB92F99093CF02C0
:101C30008091CE029091CF020E945B0E82E00C94C4
:101C4000F00D08958091CF0282FB882780F991E002
:101C500089270C940D0E81E00C940D0E80E00C94FD
:101C60000D0E6FEF7FEF80E090E00C946C2980E028
:101C700090E00E94482921E0893E9E4F09F020E033
:101C8000822F089582E090E00C943A2983E090E05E
:101C90000C943A29CF9384E090E00E943A29C82F0F
:101CA00082E290E00E943A292C2F30E0A901582BC3
:101CB000CA01CF910895CF93C92F682F84E090E097
:101CC0000E944E296C2F82E290E0CF910C944E2915
:101CD000AB01BC018FE090E00C946029AB01BC012A
:101CE00083E190E00C94602960E070E0CB010C94FB
:101CF0006E0E60E070E0CB010E94680E0C94740ED2
:101D000069EE7EEF80E090E00E946C2960E082E066
:101D100090E00E944E2960E083E090E00E944E290E
:101D20001092FA011092FB011092FC011092FD0139
:101D300060E084E090E00E944E2960E082E290E062
:101D40000E944E2960E085E090E00E944E2960E00C
:101D500086E090E00E944E296FEF87E090E00E94BD
:101D60004E2940E050E0BA0188E090E00E946029EE
:101D700060E08DE090E00E944E2940E050E0BA0122
:101D800088E190E00E94602960E087E190E00E9495
:101D90004E2940E050E0BA018CE190E00E946029B9
:101DA00060E070E080E290E00E946C2940E050E04A
:101DB000BA0188E190E00E9460290C94790E0C949D
:101DC000800E682F8EE090E00C944E290E944D21E9
:101DD000609388027093890280938A0290938B02A9
:101DE00060938402709385028093860290938702A9
:101DF000089585B7806885BF85B7806885BF0895D9
:101E000081E008950C94000F08950C94040F0C9435
:101E1000040F0C94070F0C94040F0C940B0F0C94EC
:101E2000040F0E94F90E85EC91E10E948B1F0E9425
:101E30000F0F0C940D0F0E94050F0C94040F0E94BD
:101E4000DF110E94ED030C94511C0E9438210E9466
:101E5000C4120E941F0F0E948A1A0E94C9180C9473
:101E6000090F5F926F927F928F929F92AF92BF9273
:101E7000CF92DF92EF92FF920F931F93CF93DF9356
:101E8000CDB7DEB72A970FB6F894DEBF0FBECDBF31
:101E90000E94D912C82E81110E94E60E3AE7832EC5
:101EA00032E0932E00E010E0502E802F0E940312AB
:101EB0005C01F401619071904F01682679266114EC
:101EC0007104B1F40F5F1F4F0530110569F78FEFF3
:101ED00089838A831B820E9441218160782F9D83A0
:101EE0008C8349815A816B818D810E9409043AC09B
:101EF00080918C0281FD0E940C12D12CEE24E3947F
:101F0000F12CC3018E219F21892B29F10E94020F00
:101F10008823A9F0DE825F82AE20BF2081E0AB285B
:101F200009F480E088870E9441218160782F9A8798
:101F300089874E815F8168858A850E940904000F28
:101F4000111FF801E658FD4F80819181E826F9269E
:101F5000F182E08207C0D394EE0CFF1CFFE0DF1299
:101F6000D0CFB0CF81E0C11001C080E02A960FB67B
:101F7000F894DEBF0FBECDBFDF91CF911F910F91BF
:101F8000FF90EF90DF90CF90BF90AF909F908F9099
:101F90007F906F905F9008950E94310F0E94FC180F
:101FA0000E94501C0C94FE03CF93DF930E94EE100E
:101FB000EC01811522E59207E8F5811531E59307DB
:101FC00008F0B6C0883E910528F5803E910508F0DE
:101FD000E9C0883A910570F4853A910508F07AC015
:101FE0008130910509F473C008F4D9C0049708F052
:101FF000D9C0D5C08F3B910508F0D1C0C85AD0E0F8
:10200000CC0FDD1FCB5ADE4F0990D881C02DCE01F9
:102010009464C9C0811540E5940708F069C0811532
:1020200050E4950708F060C09A9581159F4108F427
:10203000B9C0B5C0811536E5930728F5811545E58A
:10204000940708F092C0811554E5950708F087C001
:10205000AC0143705527282F26952695C115D345E9
:1020600008F06CC081E090E002C0880F991F4A958B
:10207000E2F740E2249F90011124EC01C22BD32B04
:10208000CE019C6890C081152AE5920780F48115E5
:1020900039E5930708F072C0811548E5940708F404
:1020A0007EC0D82FCC27CE01806F906A7CC090561E
:1020B0008115904208F073C08D2F8F710E9482119C
:1020C000DD27D0628F71AE01582BCA016CC081E050
:1020D00090E069C0C55AD0E0CD57DE4F8881C82F47
:1020E000D0E0CE0190645FC0DF70CE01906A5BC02B
:1020F00074E0969587957A95E1F7282F23703C2F09
:10210000337081E090E002C0880F991F3A95E2F7A2
:102110009C68AC01522B9A019C2F9F7096959695C6
:1021200050E2959FE0011124C9018C2B9D2B3BC0EF
:10213000D82FCC27CE01816F906A35C081E090E026
:1021400002C0880F991F4A95E2F750E2259F90013F
:102150001124EC01C22BD32BCE019A6824C0D82FB6
:10216000CC27CE01846F906A1EC00E9482118F71AD
:1021700090E0D82FCC27CE01906215C08F700E94BE
:10218000821194E0D695C7959A95E1F7CF70D0E08B
:10219000DC2FCC27D0699E01282BC90104C080E028
:1021A00090E001C0CE01DF91CF9108952BE4829F92
:1021B000C0011124FC012FE0729FE00DF11D1124DC
:1021C000E60FF11DEE0FFF1FEA5AFE4F8591949125
:1021D00008950E94D6100E94D40F08958238910568
:1021E00069F1B0F48133910509F46DC048F4893286
:1021F000910509F463C08A32910509F469C0089514
:102200008533910509F455C089339105B9F00895D6
:10221000833E910569F138F4803E9105B1F0823E2C
:10222000910509F10895863E9105A9F1873E910532
:10223000B9F1843E910509F064C023C02091CE021B
:1022400020FD4FC021FD4DC008958091CE0280FD3C
:1022500044C08091CF0280FF44C08091CE0284FDB3
:1022600042C083EE4DC08091CE0282FF38C0F5CFD0
:102270008091CE0282FD33C08091CF0280FD31C0BB
:10228000ECCF8091CF0281FF32C08091CE0284FDDD
:102290002AC087EE35C08091CE0283FF26C0F5CFDD
:1022A0008091CE0283FD21C08091CF0281FD1FC0AD
:1022B000ECCF8091CE0285FD1CC01DC08091CE0266
:1022C00085FD19C016C08091CE0286FD16C017C0CC
:1022D0008091CE0286FD13C010C089E311C082EE4A
:1022E0000FC080EE0DC080E00BC086EE09C084EE0A
:1022F00007C089E205C085E303C08AE201C081E32B
:1023000090E008959091CE0292FF0DC0282F287181
:10231000283019F4877F846006C0282F2471243068
:1023200011F48B7F886093FF0DC0282F287128310E
:1023300019F4877E846106C0282F2471243111F49A
:102340008B7E88612091CF0220FF0DC0382F38711D
:10235000383019F4877F816006C0382F31713130F1
:1023600011F48E7F886021FF0DC0282F287128313D
:1023700019F4877E816106C0282F2171213111F463
:102380008E7E886194FD877E089580E008950C9488
:10239000310E0E94D9128FE39CE90197F1F700C03A
:1023A00000000E94D91280E00E94031280FF04C046
:1023B0000E94C7110C948E2108950C94C9110E949B
:1023C000370E811102C00E94DF0E0E94420E8093E0
:1023D0008C020E944A0E9093CF028093CE020E94FC
:1023E000DD110E94460E682F70E080E090E00E94B0
:1023F00053086091F6017091F7018091F801909176
:10240000F9010C948B08E82FF0E0EE0FFF1FE65265
:10241000FD4F808191810895089580EA8A95F1F7B2
:10242000089500C008950C940D1208950C9415128F
:102430000C9416120C9415120C941A12F894E82F9E
:10244000E295EF70F0E031A1282F2F7081E090E04D
:1024500001C0880F2A95EAF7982F9095932391A3AE
:1024600092A1892B82A3789408950F931F93CF9301
:10247000DF93C5E9D1E089918F3F11F00E941E12D0
:1024800081E0CA39D807B9F7C6E8D1E005E911E01B
:1024900089918F3F11F00E941E120C171D07C1F782
:1024A000DF91CF911F910F910895BF92CF92DF924C
:1024B000EF92FF920F931F93CF93DF938C01C62F60
:1024C000D0E0CE018B569E4F6C01FC0190819F3F66
:1024D00009F450C0B62EF894E92FE295EF70F0E0C1
:1024E00081A19F7021E030E001C0220F9A95EAF7A8
:1024F000822B81A382A12095282322A378940E9475
:102500001112E6E8F1E045E951E021E030E0E12C8C
:10251000F12C61916F3F89F0A62FA295AF70B0E0CA
:1025200090968C9190E06F7002C0959587956A9512
:10253000E2F780FD02C0C90102C080E090E0E82A15
:10254000F92A220F331F4E175F0719F7F601808112
:102550008F3F11F00E941E1261E0E114F10409F4B2
:1025600060E08B2D0E941312CC0FDD1FC00FD11F16
:10257000F982E882DF91CF911F910F91FF90EF9048
:10258000DF90CF90BF9008950E9435128AE0EAED67
:10259000F2E0DF01982F1D929A95E9F7E0EDF2E065
:1025A000DF011D928A95E9F785E00E9424130C94BF
:1025B0006503FF920F931F93CF93DF93CDB7DEB7E1
:1025C0002A970FB6F894DEBF0FBECDBF8E010F5F06
:1025D0001F4F8AE0F80111928A95E9F7F12C6F2DCF
:1025E000C8010E945512F394F5E0FF12F8CF4AE0BB
:1025F00050E0B80180ED92E00E942D29FF24F39471
:10260000009709F4F12C892B41F08AE0F801A0ED44
:10261000B2E001900D928A95E1F72F2D45E06AED29
:1026200072E080ED92E00E9425130E9467038F2DD7
:102630002A960FB6F894DEBF0FBECDBFDF91CF91C3
:102640001F910F91FF9008950895FF920F931F938C
:10265000CF93DF93F82E092F162FD72FC42F2223C5
:1026600049F081E080938F020E94412190938E0275
:1026700080938D0280918F028823D9F080918D0202
:1026800090918E020E945921059798F0EF2DF02F1E
:10269000A12FBD2F80E090E04C2F50E084179507CC
:1026A00034F4219131912D933D930196F7CF1092FF
:1026B0008F02DF91CF911F910F91FF9008950E949B
:1026C0003B230E94250F0C9447230E944B230E941A
:1026D000CC0F0C9465230E94DF200E9422230E94CD
:1026E000110F0E945F130E9465130E941B0FFBCF06
:1026F000EF92FF920F931F93CF93DF938B01682F7D
:1027000011110AC0442329F0E82FF0E0E756FC4FEE
:102710006491762F862F75C0212F30E0E82FF0E0EE
:10272000442321F0E756FC4FE491F0E046E0049F9B
:10273000C0011124CFEFD0E0BE010E9493284BEAE4
:102740004603C001479F900D1124800F911D800FFB
:10275000911D982F990F890FAE01421B530B4E9F6D
:10276000D0014F9FB00D5E9FB00D11249B2F189F7D
:10277000A0011124452F55278E01041B150B0E9F18
:10278000A0010F9F500D1E9F500D11247E01E81ACD
:10279000F108E29E8001E39E100DF29E100D1124BF
:1027A000212F3327C21BD30BCE9F9001CF9F300D1B
:1027B000DE9F300D112462307105A9F048F46115D7
:1027C000710569F061307105C9F48B2F752F0DC04B
:1027D0006430710581F058F06630710579F47E2F10
:1027E0008B2F932F0DC0832F7B2F9E2F09C08E2FF1
:1027F0007B2F952F05C08E2F732F02C07E2F852F24
:10280000692FDF91CF911F910F91FF90EF90089565
:1028100041E00E947813089508950E9408140895D5
:10282000CF93DF93762FE901682F842F0E940D1438
:10283000798368838A83DF91CF9108958091E40240
:10284000282F269530E02115310519F4817082601A
:1028500005C02532310524F0817088648093E4023C
:10286000089588E090E00C944229CF92DF92EF9295
:10287000FF926B017C010E941E14B701A60188E043
:1028800090E0FF90EF90DF90CF900C946029E4EE01
:10289000F2E083E0808311828FEF8283838314824E
:1028A00060817181828193810C9435148091E4025E
:1028B00080FF02C08695089580E008959091E80217
:1028C000933018F49F5F9093E802882351F0609151
:1028D000E4027091E5028091E6029091E7020C9487
:1028E0003514089581E00C945E149091E8029923C8
:1028F00019F091509093E802882351F06091E4021E
:102900007091E5028091E6029091E7020C943514F3
:10291000089581E00C94751470E00C94611C609132
:1029200008018091E40280FF0AC08091070123E042
:10293000829FC001112487519D4F0C948C1480916B
:10294000090190910A01891780F7E82FF0E09F01B3
:10295000220F331FE20FF31FE751FD4F1182108248
:1029600012828F5FF0CF9091E40290FF16C0909199
:10297000090120910A01921770F4E92FF0E0DF01BC
:10298000AA0FBB1FEA0FFB1FE751FD4F8183608336
:1029900042839F5FF0CF0C948F140895CF93DF9301
:1029A00000D01F92CDB7DEB79091E40290FF0AC02D
:1029B0009E012F5F3F4F0E9410144B8169818A81D5
:1029C0000E94B3140F900F900F90DF91CF91089554
:1029D000CF93DF93EC01EC81F0E0EC56FD4F449196
:1029E000E4EEF2E0628181810E94CE148C818F5FDF
:1029F0008C83DF91CF910895CF93DF93EC01E4EEC8
:102A0000F2E0438162818C810E94CE148C818F5FC1
:102A10008C83DF91CF9108950F931F93CF93DF9312
:102A200000D01F92CDB7DEB78C018091900281114A
:102A30000AC09E012F5F3F4F4FEF6FEF0E941014AF
:102A40008A8180939002F8018481813051F028F0CE
:102A5000823061F4409190020AC08091900240E07F
:102A600007C06091900240E080E003C040E080E059
:102A700060E00E94B314F801848190E0019663E065
:102A800070E00E94A72884830F900F900F90DF9131
:102A9000CF911F910F910895AF92BF92CF92DF9285
:102AA000EF92FF920F931F93CF93DF9300D01F926B
:102AB000CDB7DEB7182FF62E042FE22E9091E40248
:102AC00090FF6DC0E92FE695AE2FB0E0A656BE4F41
:102AD0008C9180939A029E7F923061F49E012F5FC9
:102AE0003F4F812F0E9410144B8169818A810E947F
:102AF000B31443C0823019F40091E7023EC086301F
:102B000019F41091E50239C08930D9F38931A9F55A
:102B1000E9518E2F8170D82EE695F0E0EC56FC4FEF
:102B2000A590B490C12CBB2460910B01C61618F57A
:102B30002C2D30E0A29EC001A39E900DB29E900D60
:102B4000112470E00E949328812FD11002C0860FBB
:102B500001C0861B90910901290F311DA901440F65
:102B6000551F240F351F27513D4F402F6F2D0E94B9
:102B70001014C394D9CF0E948F141093E502F092E1
:102B8000E6020093E702EE2051F06091E4027091BA
:102B9000E5028091E6029091E7020E9435140F90C1
:102BA0000F900F90DF91CF911F910F91FF90EF90B9
:102BB000DF90CF90BF90AF900895E4EEF2E0918166
:102BC000282F4381628188E0890F0C944C1581E0A5
:102BD0000C94DD15E4EEF2E09181282F43816281AF
:102BE00088EF890F0C944C1581E00C94EA15E4EE03
:102BF000F2E0628128E0620F08F46FEF282F438132
:102C000081810C944C1581E00C94F715E4EEF2E010
:102C1000628128E0621B08F460E0282F43818181F3
:102C20000C944C1581E00C940616E4EEF2E043811E
:102C300028E0420F08F44FEF282F628181810C9425
:102C40004C1581E00C941516E4EEF2E0438128E087
:102C5000421B08F440E0282F628181810C944C15BE
:102C600081E00C94241620E00C944C15FF920F93F5
:102C70001F93CF93DF93EC01F12C0FEF10E06091E5
:102C80000B01F616F0F4809109012F2D30E0280F8A
:102C9000311DC901880F991F280F391F27513D4F3A
:102CA00070E0C8010E94A728962F8C814091E7020E
:102CB0006091E602F99E800D11240E941014F39495
:102CC000DECF0E948F149A818C8190FF02C08F5FAB
:102CD00001C081508C83DF91CF911F910F91FF90A4
:102CE0000895AF92BF92CF92DF92EF92FF920F932F
:102CF0001F93CF93DF93FC01828180FF02C00FEF0F
:102D000001C001E010E04CE0A42E80910B011817E7
:102D100008F043C080910901C12ED12CE601C80FF3
:102D2000D11DCE01880F991FC80FD91FC751DD4F84
:102D3000198218821A8234E0E32EF12CB12C809192
:102D400092028B0D8D302CF06A2D0E948528892FE0
:102D500005C087FF03C090910B01890F082E000C5E
:102D6000990BC816D90691F48091E7028E9DA001B7
:102D70008F9D500D112455954795559547959E016A
:102D80006091E6028091E5020E941014B00EF1E01D
:102D9000EF1AF108A1F61F5FB8CF0E948F1480913F
:102DA0009202013031F4811102C080910B018150F7
:102DB00007C090E0019660910B0170E00E94A72887
:102DC00080939202DF91CF911F910F91FF90EF902E
:102DD000DF90CF90BF90AF900895CF93809109017D
:102DE00090910A01891770F4E82FF0E09F01220FFB
:102DF000331FE20FF31FE751FD4F11821082128241
:102E00008F5FF0CFC0E060910B01C617C0F5EC2FCB
:102E1000F0E070E0CF010E94A72820910901820F05
:102E200020919102022E000C330B90E0E217F30781
:102E3000CCF020910601022E000C330B2E173F0719
:102E40008CF09C01220F331F820F931F9C0127518E
:102E50003D4F4091E7026091E6028091E5020E94B9
:102E600010140BC0FC01EE0FFF1F8E0F9F1FFC0103
:102E7000E751FD4F118210821282CF5FC4CF0E94B2
:102E80008F142091050180919102820F809391020D
:102E900090910601920F9093060119165CF4082E8A
:102EA000000C990B40910B0150E0415051098417DF
:102EB00095071CF0219520930501CF9108958F92DD
:102EC0009F92AF92BF92CF92DF92EF92FF920F93B9
:102ED0001F93CF93DF938C01FC014481C42FD0E07A
:102EE0009E01DE010E94EB289B01AC010E9401299A
:102EF0006B017C01E0E2F0E0EC1BFD0BA5E5B0E02E
:102F00009B01AC010E9401294B015C019F01DF0183
:102F10000E94E3289B01AC010E940C299B01AC019B
:102F20002C0D3D1D4E1D5F1DC501B4010E94BB2827
:102F3000C22FD22F2A3228F4F3E02F9F90011124C0
:102F40000DC025E530E02C1B3109C901880F991F00
:102F5000280F391F37FF02C02F5F3F4F3595279548
:102F6000C22FC095F12C85E5E82EED1A80910B015A
:102F7000F816C8F4F1FC02C08E2D01C08D2F90917F
:102F800009012F2D30E0290F311DA901440F551FD4
:102F9000240F351F27513D4F4C2F6091E6020E94B0
:102FA0001014F394E3CF0E948F14F80184818111EF
:102FB00002C091E003C0803219F49FEF90930401A6
:102FC00090910401890FF8018483DF91CF911F91C3
:102FD0000F91FF90EF90DF90CF90BF90AF909F90B8
:102FE0008F9008950F931F93CF93DF93EC0100E030
:102FF00010E080910B01282F30E00217130724F511
:10300000909109019801290F311DA901440F551F05
:10301000240F351F27513D4F869590E04C810817AE
:1030200019071CF4442331F002C0411103C0409140
:10303000E70201C040E06091E6028091E5020E9453
:1030400010140F5F1F4FD5CF0E948F148C8190E01A
:103050000196817099278C83DF91CF911F910F91F9
:103060000895E4EEF2E080818E7F8083608171813B
:10307000828193810E94351410929B022FEF80E78A
:1030800092E0215080409040E1F700C000000C9495
:103090008F146091E402669570E04BE050E08CE0A4
:1030A00091E00E942029892B19F481E080939B02F2
:1030B0000E944121909394028093930208959091ED
:1030C000E40290FF35C09170811102C0926006C089
:1030D000853210F0986402C0880F982B9093E40218
:1030E000662351F06091E4027091E5028091E6025E
:1030F0009091E7020E9435146091E402669570E0B9
:103100004BE050E08CE091E00E942029892B19F0DF
:1031100010929B0202C00E94491881E0809396029F
:103120004091E7026091E6028091E5020C9433162B
:103130000895682F9091E402969581E0890F853279
:1031400008F081E00C945F1881E00C949918682FC6
:103150009091E40296958FEF890F09F484E20C9424
:103160005F1881E00C94A71861E00C945F18E4EEFE
:10317000F2E080818160808386950C94B418809100
:10318000E40280FD0C9431180C94B71860E00C94A4
:103190005F188091990281112EC00E94370E811113
:1031A00004C00E94DF0E0E9447140E9431146093F5
:1031B000E4027093E5028093E6029093E7026E7F4B
:1031C00061F40E9447140E9431146093E4027093EA
:1031D000E5028093E6029093E7020E941E1410928B
:1031E0009B028091E40280FF03C086950E94C6186E
:1031F00081E08093990208950F931F93CF93DF93FB
:1032000080919B02882309F485C080919A02E09105
:10321000E402E695E81BE0939502823049F4F0E081
:10322000E057FD4FE491CE2FD0E008EE14E149C005
:10323000863049F4F0E0E357FD4FE491CE2FD0E023
:103240000CEF14E13EC0893051F4E695F0E0E6570A
:10325000FD4FE491CE2FD0E006E316E132C08F306F
:1032600051F4E695F0E0E957FD4FE491CE2FD0E020
:1032700001E716E126C0853149F4F0E0EC57FD4F37
:10328000E491CE2FD0E00DEE16E11BC0883181F025
:10329000833239F4E2E8F2E0C591D4910CE015E113
:1032A00010C0843251F4C4EFD1E002EF17E109C03D
:1032B000C8E2D0E00FE517E104C0C0EDD7E00CE0B4
:1032C00014E180919602882361F0109296020E9488
:1032D000412190939402809393021092980210924D
:1032E00097020E944121E0919302F09194028E1B7B
:1032F0009F0B8F3F9F4770F4EC0FFD1FF0939402DC
:10330000E093930283E992E0F801DF91CF911F915E
:103310000F910994DF91CF911F910F910895882308
:1033200011F0FA0101C0FB010994CF93DF93C82F7C
:10333000D62F0E9456148C1740F00E9456148D17F9
:1033400020F4DF91CF910C94A4188C2FDF91CF91B2
:103350000C94B4181F93CF93DF93FB0112811111CA
:10336000C3C0EC010E944E0D8272CD3CFCE5DF072C
:1033700009F49AC0A8F5C73CECE5DE0709F476C06D
:10338000A8F4C43C9CE5D90709F45FC028F4C33C09
:10339000DC4509F457C054C0C53C9CE5D90709F485
:1033A00059C0C63CDC4509F45CC04AC0CA3CFCE5D7
:1033B000DF0709F46AC050F4C83CECE5DE0709F405
:1033C0005AC0C93CDC4509F45BC03AC0CB3C9CE523
:1033D000D90709F45FC0CC3CDC4509F460C030C0BB
:1033E000C23DFCE5DF0709F46FC088F4CF3C9CE5E3
:1033F000D90709F460C008F45CC0C03DFCE5DF07F4
:1034000009F45CC0C13DDC4509F45BC019C0C53D91
:103410009CE5D90709F460C050F4C33DFCE5DF0723
:1034200009F455C0C43DDC4509F454C009C0C63D8B
:103430009CE5D90709F455C0CE35DD4509F454C0E3
:1034400011E052C00E94BF184FC041EB58E164EA3E
:1034500078E104C044EA58E161EB78E10E948F19F9
:1034600043C044EF55E167EE75E1F8CF47EE55E113
:1034700064EF75E1F3CF42E156E163E076E1EECF30
:1034800043E056E162E176E1E9CF40E356E161E2F3
:1034900076E1E4CF41E256E160E376E1DFCF49E84F
:1034A00054E162E774E1DACF42E754E169E874E19C
:1034B000D5CF81E017C065E082E010C068E086E00B
:1034C0000DC06EE089E00AC064E18FE007C067E1EB
:1034D00085E104C088E106C062E289E10E94951995
:1034E00003C083E20E94B418812FDF91CF911F9116
:1034F000089586E090E00C943A29682F86E090E0E9
:103500000C944E2980910D038470896280930D0381
:103510000C947D1A0E94370E811104C00E94DF0EA8
:103520000E94821A0E94791A80930D03282F2695F3
:103530002695269530E02630310524F08770886284
:1035400080930D0380910D0380FF04C086958695BE
:10355000869501C080E00C949B1B20910D03822F67
:10356000869586958695482F50E04530510554F450
:103570008F5F982F990F990F990F822F8770892B42
:1035800080930D0380910D03816080930D030E9451
:103590007D1A80910D038695869586950C949B1BCC
:1035A00080910D03982F969596959695A1F0915E32
:1035B000990F990F990F8770892B80930D03887F3E
:1035C00091E009F490E080910D0390FB80F98093E5
:1035D0000D030E947D1A80910D0386958695869530
:1035E0000C949B1B80910D0380FD13C08160809320
:1035F0000D03813019F489E080930D0380910D0350
:103600000E947D1A80910D038695869586950C946F
:103610009B1B089580910D0380FF08C08E7F8093CF
:103620000D030E947D1A80E00C949B1B08958091ED
:103630000D0380FD0C940A1B0C94F21A90910D035B
:10364000892F8695869586958F5F8F7197708630C6
:1036500038F4880F880F880F892B80930D0302C0E0
:1036600090930D0380910D03887F91E009F490E021
:1036700080910D0390FB80F980930D030E947D1AC9
:1036800080910D038695869586950C949B1B8630BC
:1036900008F085E090910D039770282F220F220FDC
:1036A000220F922B90930D03987F21E009F420E0E4
:1036B00090910D0320FB90F990930D030C949B1BAC
:1036C0000E94471B80910D030C947D1A9C01FB0105
:1036D0008281882349F12E3BFCE53F07C9F040F485
:1036E0002C3BECE53E0769F02D3B3C4561F008952D
:1036F000203C9CE5390791F070F0213C3C4589F075
:10370000089585E001C080E00E94601B80E008957C
:103710000E94D01AFBCF0E94AD1AF8CF0E94171B4F
:10372000F5CF0E941E1BF2CF81E00895279A2F98B3
:1037300008952F9808958F929F92AF92BF92CF9243
:10374000DF92EF92FF920F931F93CF93DF93C82FD7
:10375000863050F4811109C080918000877F80936A
:1037600080000E94991B06C0C5E08091800088609F
:1037700080938000A0918600B09187002C2F30E0CC
:103780000E94EB2825E030E040E050E00E94BB289A
:103790000027122F232F342F012F122F232F3327EF
:1037A00080918600909187006CE070E00E949328E1
:1037B0006017710730F0C80169E070E00E9493283B
:1037C0005EC08091860090918700E0908600F09026
:1037D0008700E0918600F0918700C6E0D0E0BE014E
:1037E0000E949328060F171F211D311D4801590102
:1037F00085E0880C991CAA1CBB1C8A95D1F7C701CF
:10380000BE010E9493286F01E12CF12CA7019601C3
:10381000260F371F411D511DC501B4010E94BB2851
:1038200069017A01E0918600F0918700CA01B9012F
:103830000E9475289B01AC01DF010E9401299B01B8
:10384000AC01C701B6010E947528DC01CB012FE055
:10385000B695A795979587952A95D1F700918600FB
:103860001091870020E030E0081719072A073B076E
:1038700028F46091860070918700CB01BC017093A1
:103880008D0060938C00DF91CF911F910F91FF907D
:10389000EF90DF90CF90BF90AF909F908F90089562
:1038A00008950E94961B8AE08093800089E18093AE
:1038B00081008FEF9FEF90938700809386000C9498
:1038C0008A1A6A9A2EB12B7F3EB134604FB7F894B2
:1038D000FC01CB01880F991F680F791F6E0F7F1FA6
:1038E000E617F70789F0819198E03EB9000000C023
:1038F00087FF2EB9880F000000C000C000C02EB99D
:1039000000C09A9591F7ECCF4FBF8FE594E00197F7
:10391000F1F700C000000895CF93DF93EC01FB01A5
:103920008281882309F43CC1C430FDE5DF0760F4DF
:10393000CB3F9CE5D90788F49E0122503C452431B9
:10394000310508F02EC109C0C236EDE5DE0729F0C9
:10395000C63AFDE5DF0709F024C10E944A0E9093A4
:10396000CF028093CE02C1318CE5D80709F4C6C0DE
:1039700008F042C0C930ECE5DE0709F49BC000F551
:10398000C5308CE5D80709F485C078F4C330ECE580
:10399000DE0709F478C008F07AC0C230DC4509F0CF
:1039A000F5C08091CE028160EFC0C7309CE5D90799
:1039B00009F478C008F07AC08091CE028061E4C03A
:1039C000CD30FCE5DF0709F487C058F4CB309CE527
:1039D000D90709F479C008F07BC08091CE028860D5
:1039E0006FC0CF30FCE5DF0709F480C008F082C06B
:1039F0008091CE02877FC8C0CE3F9CE5D90709F4ED
:103A000071C000F5C531FCE5DF0709F485C068F435
:103A1000C3319CE5D90709F475C008F095C00E9430
:103A2000FB078091CE028F77AFC0CC3FFCE5DF076C
:103A3000A9F108F054C0CB3FDC4509F0A7C0809144
:103A4000CF0240C0C230EDE5DE0709F489C058F46A
:103A5000C1158DE5D80709F45AC008F069C08091F6
:103A6000CF0282602FC0C236EDE5DE0709F47CC0CC
:103A7000C63AFDE5DF0709F481C0C330DD4509F032
:103A800085C080E06EC08091CE0282607DC0809152
:103A9000CE0216C08091CE02886076C08091CF029F
:103AA00082604FC08091CE0280626EC08091CE0253
:103AB00080646AC00E94FB078091CE02806864C067
:103AC000846062C081603DC08091CE028E7F5CC008
:103AD0008091CE028D7F58C08091CE0216C0809119
:103AE000CF0218C08091CF028D7F2BC08091CE0273
:103AF0008F7E4AC08091CE028F7D46C08091CE02DB
:103B00008F7B42C08091CE02877F8B7F3DC08091AA
:103B1000CF028D7F8E7F15C08091CE0282FB22273F
:103B200020F991E0922790FB82F990FB83F92CC059
:103B30008091CF02982F909591708E7F892B90FB6A
:103B400081F98093CF0222C00E94FB078091CE02B0
:103B500087FB222720F991E0922790FB87F914C078
:103B600081E00E94E10E12C08091CE0284FB2227E8
:103B700020F991E0922790FB84F906C08091CE0253
:103B8000982F909590FB80F98093CE028091CE0281
:103B90009091CF020E945B0E0E94FB0780E001C063
:103BA00081E0DF91CF9108950F931F9341E050E0A2
:103BB00060E070E08A019B0104C0000F111F221F0A
:103BC000331F8A95D2F7C901B8010E9453081F918B
:103BD0000F910C94FB07482F50E0FA013597EF3313
:103BE000F10508F060C0EE59FF4F0C94DD280E94EB
:103BF000DF0E55C080918C02817F8E7F80938C0276
:103C000081E080939C0208950E946A0348C08091DD
:103C10008C02982F9095917090FB80F980938C0284
:103C200091113DC0897F877F10C080918C0281FBFC
:103C3000222720F991E0922790FB81F980938C0252
:103C4000992369F180918C02816080938C0227C056
:103C500080918C0282FB222720F991E0922790FB31
:103C600082F9ECCF80918C0283FB222720F991E02E
:103C7000922790FB83F9E2CF0E94FB078091CE024E
:103C800087FB222720F991E0922790FB87F9809308
:103C9000CE0205C0895301C08D510E94D41D81E020
:103CA000089580E0FACF80E0089580E008950C94B4
:103CB000551ECF93C82F80919C02882319F0813024
:103CC00031F02BC00E944E0D823249F504C00E9493
:103CD0004E0D823261F48C2F0E94571E811104C058
:103CE0008C2F0E94EB1D17C081E090E014C08C2F38
:103CF0000E94551E81110EC0C43149F018F4CB301A
:103D000049F00FC0C93219F0C83321F00AC010922F
:103D10009C0207C081E0817006C010929C0280E086
:103D200002C080E0F8CFCF910895CF93DF93863122
:103D30009C4541F5EB010E944E0D982F8A81209100
:103D4000020130910301882379F09A7A81E009F425
:103D500080E080939D02911102C069E201C065E399
:103D6000C9010E947D200AC080919D02811102C07C
:103D700069E201C065E3C9010E9488200E94900D9C
:103D800080E001C081E0DF91CF9108950F931F93F0
:103D9000CF93DF93C42FD22FFC0182818823C9F0F7
:103DA0004093A0020E94412190939F0280939E0223
:103DB00080E28C0F883008F057C0C77081E001C0E6
:103DC000880FCA95EAF7DF91CF911F910F910C945C
:103DD00067058091A002481330C080919E029091A7
:103DE0009F020E945921883C910538F510E21D0F71
:103DF000CD17B9F080E28C0F883040F4C77081E0B5
:103E000001C0880FCA95EAF70E946E05183028F5A0
:103E100081E09D2F977001C0880F9A95EAF70E9464
:103E20006705802F0E945E051830F0F4D77081E09E
:103E300001C0880FDA95EAF70AC080E28C0F88305B
:103E400098F4C77081E001C0880FCA95EAF7DF9146
:103E5000CF911F910F910C946E05802FDF91CF9120
:103E60001F910F910C945E05DF91CF911F910F91DF
:103E700008950F939C01CB01243F4CE5340731F1A9
:103E800088F4293DFCE53F07D9F02A3D4CE534078D
:103E900079F1283D3C45A9F506E221EE41EE68EDB9
:103EA0007CE52BC0263FFCE53F07E1F0A8F0273F6B
:103EB0003C4539F507E225EE46EE67EF7CE51DC08F
:103EC00007E225EE45EE69ED7CE517C006E221EE3E
:103ED00040EE64EF7CE511C007E225EE44EE65EFAD
:103EE0007CE50BC006E221EE42EE66EF7CE505C004
:103EF00008E221E045EE6AED7CE50E94C61E80E006
:103F000008C0FC018281882319F01092A00201C030
:103F100081E00F9108959093C1018093C0010895AD
:103F20009093A6028093A5020895E091A502F091D6
:103F3000A602309721F00190F081E02D099480E0F5
:103F40000895E091A502F091A602309799F0209192
:103F50002301222359F02091CE0227FF07C0DC0164
:103F60002C9111962C93119726E02C930280F381CB
:103F7000E02D099408952091A3023091A4022817FE
:103F8000390771F09093A4028093A302E091A502F7
:103F9000F091A602309721F00680F781E02D099478
:103FA00008952091A1023091A2022817390771F0DB
:103FB0009093A2028093A102E091A502F091A60243
:103FC000309721F00084F185E02D09940895FC01DB
:103FD000329680912301882331F08091CE0287FFB1
:103FE00002C09EE101C096E080E0915028F021914E
:103FF0002223D9F38F5FF9CF0895662351F12091E1
:1040000023012223E9F02091CE0227FF19C0462F79
:104010004695469546954E31E0F4677021E030E0D4
:1040200002C0220F331F6A95E2F7FC01E40FF11D75
:10403000828190E02823392381E0232B69F409C091
:10404000FC01329608962191621729F0E817F907CA
:10405000D1F780E0089581E008959C01FC0132963B
:104060009FEF80E04191461789F09F3F19F441117D
:1040700001C0982F8F5F8630A9F79F3F39F0F90173
:10408000E90FF11D97FDFA956283089508959C014B
:104090002A5F3F4FFC014281461301C01282019604
:1040A00082179307B9F70895262F2695269526950A
:1040B0002E3168F4FC01E20FF11D677021E030E061
:1040C00001C0220F6A95EAF78281282B2283089586
:1040D000262F2695269526952E3170F4FC01E20FA9
:1040E000F11D677021E030E001C0220F6A95EAF708
:1040F0002095828128232283089520912301222361
:1041000029F02091CE0227FD0C9454200C942D20F0
:1041100020912301222329F02091CE0227FD0C9427
:1041200068200C94472020912301FC013296222321
:1041300031F08091CE0287FF02C08EE101C086E09F
:10414000DF011D928A95E9F7089508950C94A52042
:1041500083E08093A7020C94A620811102C081E025
:1041600001C082E08093A7020C94A6200C94AD209D
:1041700081E08093A7020C94A6200C94B8200895A7
:104180000C94BF200C94C0200C94BF200C94BF2032
:104190000C94BF20CF930E94C6200E94D9120E9487
:1041A000C420C0E08C2F0E940312892B29F4CF5F1A
:1041B000C530C1F780E001C081E0CF910895089536
:1041C0001F920F920FB60F9211248F939F93AF936C
:1041D000BF938091A802811113C080910E0390912A
:1041E0000F03A0911003B09111034196A11DB11DC1
:1041F00080930E0390930F03A0931003B0931103C9
:10420000BF91AF919F918F910F900FBE0F901F9014
:10421000189580911603843031F10E94D9031092D1
:10422000A80220E488E190E00FB6F894A895809366
:1042300060000FBE2093600083B7817F846083BFDE
:1042400083B7816083BF7894889583B78E7F83BF5F
:104250000FB6F894A8958091600088618093600003
:10426000109260000FBE08950E94FB070C94E003BB
:1042700082E084BD93E095BD9AEF97BD80936E0078
:1042800008952FB7F89480910E0390910F03A09199
:104290001003B09111032FBF08952FB7F8946091C8
:1042A0000E0370910F0380911003909111032FBFA3
:1042B00008959C014FB7F89480910E0390910F03DD
:1042C000A0911003B09111034FBF821B930B08956F
:1042D00078941F920F920FB60F9211248F939F9391
:1042E000AF93BF9380910E0390910F03A0911003A1
:1042F000B09111030196A11DB11D80930E039093FF
:104300000F03A0931003B0931103BF91AF919F913E
:104310008F910F900FBE0F901F90189581E08093A2
:10432000E00080E28093D8001092C9008FE19EE403
:104330000197F1F700C0000087E090EBDC0180936B
:104340001F0390932003A0932103B09322039CE0CA
:1043500088E10FB6F894A895809360000FBE909303
:104360006000FFCF8091CC0208950895CF93DF9332
:1043700020912301222339F02091CE0227FF03C090
:1043800060E222E002C068E021E02093E9002FEF24
:104390003091E800215035FD06C035ED3A95F1F732
:1043A00000002111F5CF2091E80025FF1DC0EC0190
:1043B00080912301811105C040E050E068E070E089
:1043C00003C070E040E050E0CE010E94D72380910E
:1043D000E8008E778093E80080E2FE01ACEAB2E06C
:1043E00001900D928A95E1F7DF91CF910895809326
:1043F000A9027093AB026093AA02809116038430E5
:1044000001F582E08093E9008FEF9091E800815000
:1044100095FD06C095ED9A95F1F700008111F5CF55
:104420008091E80085FF0DC040E050E063E070E05F
:1044300089EA92E00E94D7238091E8008E778093EA
:10444000E8000895BC0184E00C94F721BC0183E0EE
:104450000C94F721089580911503811109C00E94E1
:1044600068250E94C5258091E20084608093E20067
:1044700008951092150308950C94BD2060911203C5
:1044800081E0611101C080E00C94A8209091160396
:1044900081E0943009F080E0609112030C94AD202B
:1044A00042E061EC81E00E94E12442E261EC82E0C2
:1044B0000E94E1249091160381E0943009F080E09D
:1044C000609112030C94B62080911803833009F494
:1044D00061C030F4813071F0823009F49AC00895DF
:1044E0008A3009F486C08B3009F46CC0893009F039
:1044F000A8C020C080911703813A09F0A2C0809122
:10450000E800877F8093E80080911B0390911C0353
:10451000892B21F460E28CEA92E003C060E080E045
:1045200090E070E00E9422248091E8008B778093D5
:10453000E800089580911703813209F082C08091CC
:104540001B0390911C03029708F07BC08091E80048
:10455000877F8093E8008091E80082FD05C080910C
:1045600016038111F8CF6DC02091F3008091F20005
:1045700090E0922B029731F48091F100813011F09C
:10458000863021F48091F1008093CC028091E80084
:104590008B7753C080911703813A09F052C0809104
:1045A0001B0390911C03892B09F04BC08091E800FC
:1045B000877F8093E8008091E80080FFFCCF8091A6
:1045C000230136C0809117038132D9F580911B03F6
:1045D00090911C03892BA9F58091E800877F809337
:1045E000E8000E94162580911903809323010C9402
:1045F000FB0780911703813221F58091E800877FC6
:104600008093E8000E94162580911A038093CD02C2
:10461000089580911703813AA1F48091E800877F83
:104620008093E8008091E80080FFFCCF8091CD026C
:104630008093F1008091E8008E778093E8000C94DD
:104640001625089584B7877F84BF0FB6F894A89580
:1046500080916000886180936000109260000FBEBE
:1046600090E080E80FB6F894809361009093610029
:104670000FBE0C94B8200E9468250E94C525E2EE6A
:10468000F0E080818460808378940C945A2887E1DC
:1046900091E00C94901F809116038530A9F48091CD
:1046A0001603853079F40E94092180911403882330
:1046B000B1F30E94CA20882391F30E94C1230E9473
:1046C000FB07EDCF0C943421089508950C946823D2
:1046D000292F332723303105C9F060F4213031050B
:1046E00081F02230310509F044C08BE390E027EBE4
:1046F00034E043C021323105E1F02232310549F185
:1047000038C082E190E022EF34E037C09927813051
:10471000910549F028F0029761F5E9E9F4E005C058
:10472000E3EBF4E002C0E7EAF4E0849190E09F015B
:1047300024C06115710541F061307105D1F489E043
:1047400090E022EE34E019C089E090E029EC34E0FA
:1047500014C06115710541F06130710551F48DE6A9
:1047600090E024E035E009C080E490E021E735E006
:1047700004C080E090E020E030E0FA013183208343
:10478000089580E189BD82E189BD09B400FEFDCFB5
:104790008091D8008F7D8093D8008091E000826066
:1047A0008093E0008091E00081FDFCCF0895CF92DE
:1047B000DF92EF92FF920F931F93CF93DF93EC0161
:1047C0008B017A010E943525811133C0E114F10477
:1047D00039F0F70180819181081B190BC80FD91F8F
:1047E000C12CD12C0115110519F18091E80085FD2E
:1047F00016C08091E8008E778093E800E114F10400
:1048000049F0F70180819181C80ED91ED182C08202
:1048100085E00FC00E943525882321F30AC08991C5
:104820008093F10001501109FFEFCF1ADF0ADACFB0
:1048300080E0DF91CF911F910F91FF90EF90DF907B
:10484000CF90089520911D0330911E03261737073E
:1048500048F06115710539F42091E8002E77209316
:10486000E80001C0B901FC0120E06115710579F192
:10487000809116038823F1F18530F1F18091E800F1
:1048800083FD3CC08091E80082FD2EC08091E8004D
:1048900080FFEBCF2091F3008091F20090E0922B0B
:1048A0006115710551F08830910538F421912093FC
:1048B000F100615071090196F3CF21E0089709F0EA
:1048C00020E08091E8008E778093E800CECF211120
:1048D000CFCF0AC080911603882361F0853061F044
:1048E0008091E80083FD0AC08091E80082FFF2CF4A
:1048F00080E0089582E0089583E0089581E00895BE
:1049000020911D0330911E032617370748F06115CB
:10491000710539F42091E8002E772093E80001C05A
:10492000B901FC0120E06115710591F18091160338
:10493000882309F440C0853009F43FC08091E80025
:1049400083FD3DC08091E80082FD2FC08091E8008A
:1049500080FFE9CF2091F3008091F20090E0922B4C
:104960006115710559F08830910540F42491209328
:10497000F1003196615071090196F2CF21E008975C
:1049800009F020E08091E8008E778093E800CBCF9B
:104990002111CCCF0AC080911603882361F08530A5
:1049A00061F08091E80083FD0AC08091E80082FFF9
:1049B000F2CF80E0089582E0089583E0089581E0D9
:1049C0000895982F973068F59093E900981739F07B
:1049D0007091EC002091ED005091F00003C0242F65
:1049E000762F50E021FD02C09F5FECCF3091EB00AD
:1049F0003E7F3093EB003091ED003D7F3093ED0032
:104A00003091EB0031603093EB007093EC00209319
:104A1000ED005093F0002091EE0027FDE5CF80E0FF
:104A200008958F708093E90081E0089580911703C5
:104A300087FF11C08091E80082FD05C080911603B8
:104A40008111F8CF11C08091E8008B770BC0809165
:104A50001603882349F08091E80080FFF8CF809109
:104A6000E8008E778093E80008952091E40030916B
:104A7000E50095E64091EC00842F817040FF23C053
:104A80008091E80080FD1DC080911603882399F075
:104A9000853099F08091EB0085FD11C04091E400D4
:104AA0005091E5002417350729F3915011F09A0130
:104AB000E1CF84E0089582E0089583E0089581E0E5
:104AC000089580E008954091E80042FFDDCF089509
:104AD0000E94D6250E94DE25E0EEF0E08081816014
:104AE0008083E8EDF0E080818F77808319BCA7EDAB
:104AF000B0E08C918E7F8C9380818F7E808310922A
:104B0000150308950F931F93CF93DF930E94D6252B
:104B10000E94DE25C8EDD0E088818F778883888168
:104B20008068888388818F7D888319BC10921603E2
:104B300010921203109214031092130300EE10E06F
:104B4000F80180818B7F808388818160888342E047
:104B500060E080E00E94E124E1EEF0E080818E7F61
:104B60008083E2EEF0E080818160808380818860D4
:104B70008083F80180818E7F808388818061888333
:104B8000DF91CF911F910F910895E8EDF0E08081C2
:104B90008F7E8083E7EDF0E080818160808384E018
:104BA00082BF81E0809315030C948225E8EDF0E04C
:104BB00080818E7F80831092E20008951092DA0047
:104BC0001092E10008951F920F920FB60F921124D8
:104BD0002F933F934F935F936F937F938F939F9305
:104BE000AF93BF93EF93FF938091E10082FF0BC0DF
:104BF0008091E20082FF07C08091E1008B7F80936B
:104C0000E1000E9459288091DA0080FF1FC0809146
:104C1000D80080FF1BC08091DA008E7F8093DA007D
:104C20008091D90080FF0DC080E189BD82E189BDFE
:104C300009B400FEFDCF81E0809316030E942B2271
:104C400005C019BC109216030E9439228091E10020
:104C500080FF19C08091E20080FF15C08091E200C2
:104C60008E7F8093E2008091E20080618093E20079
:104C70008091D80080628093D80019BC85E0809331
:104C800016030E943E228091E10084FF30C0809193
:104C9000E20084FF2CC080E189BD82E189BD09B4B6
:104CA00000FEFDCF8091D8008F7D8093D800809149
:104CB000E1008F7E8093E1008091E2008F7E8093FF
:104CC000E2008091E20081608093E2008091120313
:104CD000882311F084E007C08091E30087FD02C0C3
:104CE00081E001C083E0809316030E9446228091F8
:104CF000E10083FF29C08091E20083FF25C08091FD
:104D0000E100877F8093E10082E080931603109298
:104D100012038091E1008E7F8093E1008091E20098
:104D20008E7F8093E2008091E20080618093E200B8
:104D300042E060E080E00E94E1248091F000886021
:104D40008093F0000E943C22FF91EF91BF91AF91C0
:104D50009F918F917F916F915F914F913F912F9193
:104D60000F900FBE0F901F9018951F920F920FB6C5
:104D70000F9211242F933F934F935F936F937F93E1
:104D80008F939F93AF93BF93CF93DF93EF93FF9353
:104D9000C091E900CF708091EC00D82FD17080FDD8
:104DA000D0E81092E9008091F000877F8093F000B6
:104DB00078940E94F9261092E9008091F0008860B2
:104DC0008093F000CD2BCF70C093E900FF91EF915D
:104DD000DF91CF91BF91AF919F918F917F916F9113
:104DE0005F914F913F912F910F900FBE0F901F90A9
:104DF00018951F93CF93DF93CDB7DEB7AA970FB661
:104E0000F894DEBF0FBECDBFE7E1F3E08091F10083
:104E1000819323E0EF31F207C9F70E946422809169
:104E2000E80083FF2EC18091170390911803492F4A
:104E300050E04A30510508F024C1FA01EF55FF4F08
:104E40000C94DD28803821F0823809F01AC108C09E
:104E50008091130390911403992389F082600FC00D
:104E600080911B038F70873008F00BC18093E9009D
:104E70008091EB0085FB882780F91092E9009091E2
:104E8000E800977F9093E8008093F1001092F10082
:104E9000D1C0282F2D7F09F0F4C0882319F082306B
:104EA00061F0EFC080911903813009F0EAC09330BE
:104EB00009F080E0809314032EC0809119038111C2
:104EC0002AC080911B038F702FEF280F263008F027
:104ED000D8C08093E9002091EB0020FF1CC09330E4
:104EE00021F48091EB00806214C09091EB009061FE
:104EF0009093EB0021E030E0A90102C0440F551F60
:104F00008A95E2F74093EA001092EA008091EB0064
:104F100088608093EB001092E9008091E800877F21
:104F20008093E8000E941625ACC08111AAC01091A0
:104F300019031F778091E3008078812B8093E30031
:104F40008091E800877F8093E8000E941625809179
:104F5000E80080FFFCCF8091E30080688093E3004D
:104F6000111102C082E001C083E08093160389C062
:104F70008058823008F085C08091190390911A03FF
:104F80008C3D53E0950779F583E08A838AE2898333
:104F90004FB7F894DE01139620E03EE051E2E32F94
:104FA000F0E050935700E49120FF03C0E295EF70CA
:104FB0003F5FEF708E2F90E0EA3010F0C79601C08F
:104FC000C0968D939D932F5F243149F74FBF8091F9
:104FD000E800877F8093E8006AE270E0CE010196E6
:104FE0000E94222416C060911B0370911C03AE0125
:104FF0004F5F5F4F0E946623BC01892B09F441C0BB
:105000009091E800977F9093E80089819A810E94AF
:1050100080248091E8008B778093E80032C080384C
:1050200081F58091E800877F8093E80080911203EA
:105030008093F1008091E8008E7772CF811121C0BA
:105040008091190390911A0399270297D4F48091C3
:10505000E800877F8093E800809119038093120312
:105060000E94162580911203811106C08091E300F1
:1050700087FD02C081E001C084E0809316030E9496
:1050800050228091E80083FF0AC08091E800877F6A
:105090008093E8008091EB0080628093EB00AA96F9
:1050A0000FB6F894DEBF0FBECDBFDF91CF911F9139
:1050B00008950895CF93809116038823A1F0C0919D
:1050C000E900CF709091EC00892F817090FD80E80D
:1050D000C82B1092E9008091E80083FD0E94F92618
:1050E000CF70C093E900CF910895DB018F939F9318
:1050F0000E940129BF91AF91A29F800D911DA39F96
:10510000900DB29F900D1124089587FB082E06265E
:1051100087FD819567FD61950E9414290EF4919594
:1051200007FC81950895AA1BBB1B51E107C0AA1F6C
:10513000BB1FA617B70710F0A61BB70B881F991F38
:105140005A95A9F780959095BC01CD01089597FBDC
:10515000072E16F4009407D077FD09D00E949328FB
:1051600007FC05D03EF4909581959F4F089570956A
:1051700061957F4F0895A1E21A2EAA1BBB1BFD016A
:105180000DC0AA1FBB1FEE1FFF1FA217B307E40726
:10519000F50720F0A21BB30BE40BF50B661F771F7E
:1051A000881F991F1A9469F760957095809590955E
:1051B0009B01AC01BD01CF010895EE0FFF1F0590CB
:1051C000F491E02D09940E94EB28332312F48A1BFA
:1051D0009B0B0C94FC28A29FB001B39FC001A39F1E
:1051E000700D811D1124911DB29F700D811D112420
:1051F000911D08950E94EB28B7FF0895821B930B21
:1052000008950E94EB28A59F900DB49F900DA49F38
:10521000800D911D11240895B7FF0C9401290E945F
:105220000129821B930B0895991B79E004C0991FF3
:10523000961708F0961B881F7A95C9F780950895F0
:10524000FC014150504030F001900616D1F73197E3
:10525000CF010895882799270895FB01DC0104C038
:105260008D910190801921F441505040C8F7881B5E
:10527000990B0895F999FECF92BD81BDF89A9927AF
:1052800080B50895A6E1B0E044E050E00C947429A4
:10529000A8E1B0E042E050E00C947429262FF9997F
:1052A000FECF92BD81BDF89A019700B4021639F085
:1052B0001FBA20BD0FB6F894FA9AF99A0FBE089556
:1052C0000396272F0E944F290E944E29252F0E94C6
:1052D0004F29242F0C944F290196272F0E944F29E4
:1052E0000C944E29DC01CB01FC01F999FECF06C0DC
:1052F000F2BDE1BDF89A319600B40D924150504094
:08530000B8F70895F894FFCFFF
:10530800C8005802010102000C000C0C01191A1BFC
:105318001C1D1E1F202122B221B6212A222622224C
:1053280022B52101E200E900EA00B500B600B700A5
:10533800CD008301CC008A0192019401210223024D
:1053480024022502260227022A02B300B4006F00B5
:105358007000818283E200E900EA00B500B600B778
:1053680000CD008301CC008A01920194012102231F
:105378000224022502260227022A02B300B4006F83
:10538800007000818283F0F1C66766369431F73584
:10539800349796333290919293950001020202025B
:1053A8000606060909090909090F0F0F0F0F0F153E
:1053B8001515181919191919191919191923240062
:00000001FF
